:030000000219FDE5
:03000B000200A848
:03002B000201557A
:03005B000202DEC0
:030073000202CBBB
:1000800002030406080C10182030406080040608A3
:100090000C10182030406080A0C00003070F1F051F
:1000A000050D050205030302C2AFC0D0C0E0206207
:1000B00014E5256009E473E525F4F58AD262D0E001
:1000C000D0D0D2AF3285268AC262E526F4602AD02B
:1000D000E0D0D0C295C294C293D2AF32C295C2943E
:1000E000C293206F0D20660A7405D5E0FDE57BF410
:1000F0005290D0E0D0D0D2AF32758A00C28DD26299
:1001000001F201B7306805206602D29501B7306868
:1001100005206602D29401B7306805206602D293AA
:1001200001B7D29230680A2066077403D5E0FDD289
:100130009501B7D29130680A2066077403D5E0FDB7
:10014000D29401B7D29030680A2066077403D5E0D4
:10015000FDD29301B7C2AFC2AD53E6EFC0D0C0E04D
:10016000D2D3D2AFC2CEE52A6007207449152A2126
:10017000B67800790020742EE580307E01F430E7F7
:100180000278FF53DACF207E0343DA20307E034328
:10019000DA10C2D8C271E580307E01F430E702790E
:1001A000FFC3E89970CB306103752A18207403757A
:1001B0002A18885CD27020740DE52B6004152B2161
:1001C000C643DA01C2D82070024139A85C2061021E
:1001D000C270207431C3E894F0400374F0F8E8C4AE
:1001E000540F28F87984B703024106C313C3138759
:1001F00021200802C313200A06C3C898F841062824
:10020000F8500374FFF8C3E895655003E565F88876
:1002100022E52D54066022206B1FE536C333C3331D
:10022000F8E564C313C313F9C3952240028922E899
:100230002522F52250037522FF852224A824C3E538
:100240002495614002A8618825E5667002417DC35E
:10025000E8AA669A5003E8FAE4F9EAC333FBE568D2
:10026000F45B29400D2567F8E56760021567400BD0
:10027000417D0AC3E5679A5002056778FF8826C367
:10028000E52594404002D26420CF0AD0E0D0D0438C
:10029000E610D2AD32C2CF053A7801E52A600530CA
:1002A0007402152AC3E55C94014005755F0041C1E5
:1002B000756000756900E55F2401F55F5003755FA7
:1002C000FFD0E0D0D043E610D2AD32C2AF53E67FCC
:1002D0007592FA7593FFC260759104D2AF32C2AFC6
:1002E00053E6EFC2ADC0D0C0E0C0F0D2D3D2AFA8C9
:1002F000FBA9FCC2D8307102614553DACF207E03DE
:1003000043DA10307E0343DA20D271E580307E017B
:10031000F420E702611C88278928A17253DACF20D4
:100320007E0343DA20307E0343DA10C2D8C2713034
:100330007402A15E7800E580307E01F430E702A10E
:100340005E885CA14653DACF207E0343DA20307EFC
:100350000343DA10C271206102811E53DACF207E7E
:100360000343DA10307E0343DA20C2D8D2718857B3
:100370008958C3E89555F8E99556F97B007E087AC7
:1003800000C3E8948CE994005005755B00811088E7
:100390002178A2E6A8216055C3E894C8E9940050EA
:1003A00008E4D2E4FB7A0A61EBC3E89468E99401BB
:1003B0005008E4D2E3FB7A0F61EBC3E894D0E994F0
:1003C000025008E4D2E2FB7A1E61EBC3E894A0E994
:1003D00094055008E4D2E1FB7A3C61EBC3E89498C1
:1003E000E994085008E4D2E0FB7A787E00C3E895EF
:1003F00059FCE9955AFD30E70AECF42401FCEDF4D0
:100400003400FD755B00C3EC9AED9E5003755B01F3
:100410008859895A8557558558567802A146C3E8A8
:100420009527F8E99528F9307C02A12A307B02A1B2
:100430002A307A02A1232075028141E9FDE8FC817E
:1004400060E9C313F9E813F8307902A123E9C31373
:10045000F9E813F8307802A123E9C313FDE813FC8F
:1004600020612CC3EC941CED940240028177ED7066
:0F0470001EC3EC94C850180529E5297002152900
:10047F00C3E529940A5002A15E755C00D270A15E9B
:10048F00E529600215297888E6F97400207F08783D
:10049F0096B90302789EE624FAFEE43400FFC3EC1B
:1004AF009EFCED9FFD9208B90310A208500720761D
:1004BF0009D27681C9307602C276A2085016B903E6
:1004CF000DECF42401FCEDF43400FD0204E378009C
:1004DF007900A12AB90315EC33FCED33FDC3EC947D
:1004EF000AFCED9400FD50047C007D00C3EC94FFEA
:1004FF00ED9400400678FF7900A12AEC8572F0A4F4
:10050F00C5F0A2F733F87900400302054678FF796A
:10051F0000020546E9C313F9E813F8307C0EE960D1
:10052F000278FFC3E81338F8E43400F9C3E894FF06
:10053F00E99400400278FF885CD270206102A15ECE
:10054F00741FF4552F4BF52FC274EB7002D27475D4
:10055F002A18307403752A0A306102A172207403BD
:10056F0053DAFE207403752B06D0F0D0E0D0D0D232
:10057F00AD43E6103279010205A279030205A27993
:10058F000A0205A2791E0205A279640205A279C8A2
:10059F000205A27817E4D5E0FDD8FAD9F6227A142D
:1005AF007B780205C97A107B8C0205C97A0D7BB462
:1005BF000205C97A0B7BC80205C97902E4D291D52D
:1005CF00E0FDD294D5E0FDC294D5E0FDC291D5E017
:1005DF00FDE920E002D29530E002D293E573D5E039
:1005EF00FDE920E002C29530E002C2937496D5E097
:1005FF00FDD9C9EAF8D5E0FDD8FBDBBED29122C305
:10060F007C007D0075F00005F0EA33FAEB33FB5008
:10061F00F6EB13FBEA13FAC3E9FFE8FEE89AF8E9F1
:10062F009BF95004EFF9EEF8B3EC33FCED33FDD545
:10063F00F0DFEDF9ECF822E889F08A20D2D4F8A99E
:10064F00F07B0030F70B7BFFF42401F8E9F4340062
:10065F00F9E88520F0A4ADF0F8E98520F0A4AFF01B
:10066F00FEED2EF974003FFA7C04C3EA13FAE91386
:10067F00F9E813F8DCF48BF030F70AE8F42401F80A
:10068F00E9F43400F9E889F0C2D4F8A9F02222C3C2
:10069F00E54113F9E54013F8C3E54498F8E54599AA
:1006AF00F9500CC3E89480E994FF40160206D5C3B5
:1006BF00E8947FE9940050030206D5787F79000211
:1006CF0006D5788079FF8849894A22E5492546F879
:1006DF00E54A3547F9854A20E4300701F43548FAF1
:1006EF0030E709C3EA94F04015020713C3EA940FE9
:1006FF00500302071378FF79FF7A0F020713780070
:10070F0079007AF0C3E5249561500AC374019524EA
:10071F00500B020731E54A20E70E020731E54A3058
:10072F00E706884689478A482278A5E6FAC3E5494D
:10073F0033F8E54A33F9D146E930E70BC3E8948043
:10074F00E994FF4013E16BC3E8947FE994005002F2
:10075F00E16B787F7900E16B788079FFE820E7150E
:10076F00C3E52398F84009C3E894014003020792B8
:10077F007801020792E8F424012523F840030207C9
:10078F009278FF884B2278A6E6FAA847A948D14667
:10079F00E930E70CC3E89401E994FF40160207C65D
:1007AF00C3E894FFE9940050030207C678FF79006D
:1007BF000207C6780179FFE920E715C3E54B98F8E2
:1007CF004009C3E8940140030207ED78010207EDE9
:1007DF00E8F42401254BF840030207ED78FF882445
:1007EF002278FFC26420693D206A12D264C3E541BA
:1007FF00940A4009C3E52594405002C26479A1E7E9
:10080F006023E541601F74FF8541F0848539F03026
:10081F006A0375F005A4F8C5F0600278FFC3E89588
:10082F00645002A864886322C3E5409440E5419474
:10083F0001E5635003140148046002F563220208C6
:10084F00502275E890227883E6FFE5E820ECF7A8C0
:10085F00BDA9BE0570C3E57094084052757000E9DC
:0D086F00FA79A0E76044EA7007E571601BAC
:10087C0002088BC3E895716010E5715006600C148A
:10088C000208970460F9020897E571F571C3946D3D
:10089C00401B7561C0C394044013756180C39404FC
:1008AC00400B756140C39404400375610075BB0631
:1008BC0022E561F460020561E570B4070375BB10B5
:1008CC0022743279A787F0A4C5F0A2F733F8C3E8F5
:1008DC0095614002A861882288248825882688642E
:1008EC00227540007541F022C2AF75C820A8CCA972
:1008FC00CDAA3A30CF010A75C824D2AFAB3BAC3C81
:10090C00883B893CC3E89BF8E99C206908F930676F
:10091C00024100215DAD3D8A3DF9EA9DFA60047803
:10092C00FF79FFAE3EAF3F8B3E8C3FA83BA93CC34B
:10093C00E89EF8E99FF9C3E54113FBE54013FAE89B
:10094C002AF540E93BF54150067540FF7541FF2102
:10095C00A7AA40AB41AC40AD417E047F02C3EB94EF
:10096C000440021E1FC3EB940840021E1FC3ED136C
:10097C00FDEC13FCDEF7C3EA9CFAEB9DFBEF600980
:10098C00C3E913F9E813F8DFF7EA28FAEB39FB8A25
:10099C00408B4150067BFF8B408B41C3EB94025044
:1009AC0002D2673069047F0321D27892E6FFC3E557
:1009BC0037948240110FC3E53794A040010FC3EF69
:1009CC00940640027F057E02E541C4540FF9E541CF
:1009DC00C454F0F8E540C4540F28F8C3E89EFAE973
:1009EC009400FB4009C3EA9402EB940050047A0291
:1009FC00E4FB414CAA40AB41EBC4FEEAC4540F4E9D
:100A0C00FCC3EA9CFAEB9400FBC3E813C313F8EAAB
:100A1C0028FAEB3400FB8A408B41C3EB9402400272
:100A2C00C2677802EBC4FE7B00EAC4540F4EFAC3D3
:100A3C00EA98FA4005C3940250027A027892E6FFD3
:100A4C00306002414C855192855293D26043E680CE
:100A5C00C3E49AF8E49BF930670241D8E8FAE9FB61
:100A6C00D3E913FDE813FC88518952C3EF9403605A
:100A7C0038EF20E00DE82CF8E93DF9ECFAEDFB023B
:100A8C000AA1E828F8E939F9C3E82402F8E93400A6
:100A9C00F97AFE7BFFC3EF9403400E8A538B548884
:100AAC004D894E8C4F8D50610C885389548A4D8BD7
:100ABC004E8C4F8D503069127553F07554FF754F35
:100ACC00F07550FF7551F07552FF610CE8FAD3E8E0
:100ADC0013FC8851C3EF94036020EF20E007E82C4F
:100AEC00F8ECFA41F8E8282402F87AFEC3EF9403F4
:100AFC0040088A53884D8C4F610C88538A4D8C4F1B
:100B0C00E568C3335002646BF5683060026116759A
:100B1C003402D26043E680E52D54066034A840A927
:100B2C0041C3E913F9E813F8C3E913F9E813F830F2
:100B3C006904E92440F9C2AF53E67F759100C3E420
:100B4C0098F594E499F595759104D26043E680D2BA
:100B5C00AF22D265754300752000306C03752040C0
:100B6C00020B7DD265754300752040306C037520F7
:100B7C000078017901206720E52D54066002C265DA
:100B8C007914E541C313700104F8C394144002783E
:100B9C0014306904781B791B206010E543600C301D
:100BAC006903D53404D26D811F711E0543E59B5436
:100BBC0040B52002810930690908C3E89940011841
:100BCC0061A420650A08C3E8994002617D61A4C252
:100BDC0065C2AF53E67F759100306712759400754E
:100BEC0095FE759104D26043E680D2AF617DAE4034
:100BFC00AF41C3E49EF594E49FF59561EEC3E533F4
:100C0C0094015002617D306502617DD802811D61C5
:100C1C00A4C26DC2AF53E67F759100855394855481
:100C2C0095759104854D92854E93D26043E680D2A2
:100C3C00AFE52D54066008206A020533020C5B30C8
:100C4C006D0D206C0A206507158115810214F122A7
:100C5C0078003064053065027801E53775F007A43B
:0F0C6C00F9E5F028F5F0E9A2F013A2F113A2F2D6
:100C7B0013F537C394785003753778C3E537953838
:100C8B004008D266C295C294C293306002819585AA
:100C9B004F92855093D26043E68022207D16C2AFDF
:100CAB00754202D291C292306202D293D2AF759F3B
:100CBB0011020E95C2AF754202D291C29030620200
:100CCB00D295D2AF759F11020E95307243207D20C5
:100CDB00C2AF754203900133757B02C293D2903041
:100CEB006204D29481F3C291D2AF759F01020E952B
:100CFB00C2AF754203900133757B02C295D292301D
:100D0B006204D294A113C291D2AF759F21020E95AA
:100D1B00207D17C2AF75420390010EC29330620261
:100D2B00D294D2AF759F01020E95C2AF754203905C
:100D3B00010EC295306202D294D2AF759F21020E82
:100D4B0095207D16C2AF754204D292C290306202DA
:100D5B00D294D2AF759F21020E95C2AF754204D2C9
:100D6B0090C292306202D294D2AF759F01020E955F
:100D7B00307243207D20C2AF754205900122757BF6
:100D8B0004C294D291306204D295A199C292D2AF8F
:100D9B00759F11020E95C2AF754205900144757B8C
:100DAB0001C294D291306204D293A1B9C290D2AF56
:100DBB00759F11020E95207D17C2AF7542059001EC
:100DCB0004C294306202D295D2AF759F11020E9578
:100DDB00C2AF754205900118C2943062EBD293D228
:100DEB00AF759F11020E95207D16C2AF754206D2CC
:100DFB0090C291306202D295D2AF759F01020E95CF
:100E0B00C2AF754206D292C291306202D293D2AF78
:100E1B00759F21020E95307243207D20C2AF754223
:100E2B0001900144757B01C295D292306204D2933A
:100E3B00C13FC290D2AF759F21020E95C2AF7542D2
:100E4B0001900122757B04C293D290306204D2953B
:100E5B00C15FC292D2AF759F01020E95207D17C262
:100E6B00AF754201900118C295306202D293D2AF96
:100E7B00759F21020E95C2AF754201900104C2937A
:100E8B00306202D295D2AF759F01C26622900102E9
:100E9B00757B00C295C294C293D292D291D290C26A
:100EAB006222788076FF0876FF0876FF0876FF08C7
:100EBB00760308760408760A087601087601087628
:100ECB0001788C76010876FF0876FF0876FF0876A6
:100EDB00FF0876FF0876030876FF0876FF0876FF93
:100EEB000876250876D00876FA0876FA087604088C
:100EFB0076FF08760108760008767A0876FF087682
:100F0B0001087601087600087603087600227887B8
:100F1B00E6FFC2727888E6C394036008C27DE630B0
:100F2B00E102D27DC27E7889E630E102D27EC3EF48
:100F3B0094026008758E01D273020F4C758E00C23D
:100F4B0073227880E6149000809378A5F67881E67A
:100F5B00149000809378A6F67886E61490008D9313
:100F6B0078A7F67886E6F539C394025003753902F3
:100F7B00789CE67538FFB402037538A0B40303758B
:100F8B00388278A3E61490009A93F566D1982222C2
:100F9B007896E6FA7897E6FB7888E6B40305C3EB18
:100FAB00940EFB307F047A007BFFC3EB9AFCC39457
:100FBB008250027C827572000572EC8572F0A4C3BC
:100FCB00E5F0947D40F222D27FF19B1205937A00DB
:100FDB007B007C10120589E55C2AFA74003BFBDC74
:100FEB00F37C04C3EB13FBEA13FADCF7FEC27FF1CD
:100FFB009B22E5EF20E6037520000520903FFFE5DF
:10100B0020146006901DFF1460009304600375EFBD
:10101B001253D9BF7581C043FF8012058475EF024F
:10102B0043B203E5B3240220E70DF521E5E320E00D
:10103B00068521B343E301120E987580FF75A4005A
:10104B0075F19075D47F75908775A5BF75F2BF75D7
:10105B00D50075A60175E241120E98E4F8F6D8FD9D
:0D106B00756801120EAD121542789886735B
:10107800753001C2AF12059D1205AD120593120518
:10108800B41205931205BB12059312165B12059D47
:1010980012059D120598C2AF78FA79FA308707D9F8
:1010A800FBD8F7021C00120F19120F4D120F9A12DB
:1010B8000F9B78988673120E98758810758902753B
:1010C800C82475910475D84075A82275B80275E6CC
:1010D80090759B80759D0075D10E75BC5875BB06C3
:1010E80075BA1175E880120584D2AF12084D7536AD
:1010F8000053DACF207E0343DA20307E0343DA1030
:1011080043DA01C2D8C27112059DD2617B037A0C01
:10111800E55B70077A0CDB0302109E1205932070C2
:101128000302109EC270E55CC3940240E1E52F54AF
:101138001F855E5DF55EB55DD5DAD5C26153DACF40
:10114800207E0343DA20307E0343DA10C2D8C2710E
:1011580078A2E67008D274E52F54E0F52FC27575B1
:101168002900120598307409C3E529940A4002D26F
:101178007512058978023074027800C3E55C9840DE
:10118800F0C2AF1205AD1205AD1205ADD2AF120512
:101198009D754C007888E6B4030241811205897870
:1011A8008CE6C394015003021281E530C3940150C8
:1011B80003021281207435C3E55C94FF50030212C8
:1011C80081C2AF1205C2D2AF120598C3E55C940183
:1011D80050EFC2AF1205AD12058E1205ADD2AF1297
:1011E8000598C3E55C94FF40E90216E07F05D27FCD
:1011F800120F9B120598C2AFC27F120F9BAE5CC341
:10120800E55C947FD2AF407B120584C2AF1205C261
:10121800D2AFDFDA120FD2C3EE94057897F6120533
:101228009D1215841216637F0AD27F120F9B120536
:1012380098C2AFC27F120F9BAE5CC3E55C947FD2AD
:10124800AF50E4120584C2AF1205AD12058E120527
:10125800ADD2AFDFD4120FD2EE24037896F6120582
:101268009D121584121692120598120F9BC3E55C05
:1012780094FF500221BC0216E0C3E55C954C400384
:10128800855C4C12059878017988E7B403027805E3
:10129800C3E55C984002219CC2AF1205C21205C288
:1012A8001205C2D2AF12059D753000E4F531F53252
:1012B8000531E531F4703F0532789AE67819146003
:1012C80012783214600D787D14600878FA1460037F
:1012D800753200C3E53298401D120E981205841528
:1012E8003275310078998673C2AF1205C2D2AF78D1
:1012F80098867312059812058EE52A7005307402D7
:10130800019E78012074027806C3E55C9840A178B4
:1013180088E6C394036003120598E52A7003021057
:101328009EC2AF120E98E4F522F523F524F525F5B3
:1013380026F567D2AF7885E6C333F565E4F544F55D
:1013480045F546F547F548F570F52CF52DF5377553
:10135800700875BB10120584120851E5E820ECFBF3
:10136800A8BDA9BEE97001F8887112085575700802
:1013780075BB10120F19C2AF7561FF1208CD852217
:1013880061852262852263D2AF75220175240175B9
:101398002501752601856069756A017888E6B403B8
:1013A80007C27D307602D27DD268D26975330012C9
:1013B8000DF2120E211208ED1208F41208ED1208AF
:1013C800F41208ED120B6F12069D120C5C120CA69B
:1013D8001208F4120B5E306E0312069E2067031289
:1013E80007F0306703120837120C5C120CD512088C
:1013F800F4120B6F306E031206DA120C5C120D4CED
:101408001208F4120B5E306E03120738120C5C12CD
:101418000D7B1208F4120B6F306E03120795120C35
:101428005C120DF21208F4120851120B5E120C5CD9
:10143800120E211208551208F430692F856461854F
:101448006462856069756A0179187A0CC3E5339915
:10145800400CC269D26A8A357561FF021473C3E50C
:0E1468005C940140030213CC0214F9306A1D9B
:10147600206C1AE535147006C26AD26B61CCF5355C
:10148600C3E55C940140030213CC0214F9753600DF
:10149600788279A4E760027803C3E55F98505430F8
:1014A6007404E52A604D7888E6B40317207D05208C
:1014B600760781C930760281C9206C07D26C8564B3
:1014C60061810B78F0306C058564617820C3E54155
:1014D60098500261CC306C1BC26CC27D307602D251
:1014E6007DD26A75351285646161CC0536E55C602E
:1014F6000281FC753600C2AF120E987887E6FE763A
:1015060002120F197887EEF6E4F522F523F524F595
:1015160025F526F565752C00752D00D2AF120598B8
:10152600120E9878A4E66006C292C291C2903074F8
:1015360009C3E53694044002019E41B3901A0D7822
:10154600201215C6E520B45A0CA31215C6E520B420
:10155600A503021564120EAD121584021583901AA6
:101566000378807B0A1215C6A308DBF9901A0F7858
:101576008C7B191215C6A308DBF9901A2822C2AF74
:101586001216051215DF901A00740E1215CBA374ED
:10159600061215CBA374151215CB901A0378807B0F
:1015A6000A1215CAA308DBF9901A0F788C7B191258
:1015B60015CAA308DBF91216181215F6901A282276
:1015C600E493F622E6438F01538FFD75EF0275B75C
:1015D600A575B7F1F0538FFE22438F02438F017535
:1015E600EF0275B7A575B7F1901A0DF0538FFC226F
:1015F600901A0D745AB1CB901A0E74A5B1CB227AFB
:101606003079D07820901A40B1C6E520F709A3DAE0
:10161600F7227A3079D0901A40E7B1CB09A3DAF9EC
:1016260022AB74A875BB01027984BB02027985BB23
:1016360003027986BB04027992BB05027987BB0651
:101646000279A3BB0702799CBB08027988BB090211
:101656007989E8F7227C0512059DDCFB22C2AF12D0
:1016660005AD1205B41205BB1205C212058E120590
:10167600AD1205B41205BB1205C212058E1205ADD8
:101686001205B41205BB1205C2D2AF22C2AF1205B3
:10169600C21205BB1205B41205AD12058E1205C2A3
:1016A6001205BB1205B41205AD12058E1205C21243
:1016B60005BB1205B41205ADD2AF22AE74AF75C22A
:1016C600AF1205AD1205AD1205AD12058EDEF21292
:1016D60005C212058EDFF8D2AF22D163D15BD15B92
:1016E600757401757501757600D1C17C05AD5C1206
:1016F600059DC3ED955C70F5C3E55C9401400AC396
:10170600E55C94FF403202171CD127B184D163C235
:10171600AF75EF12D15BDCD50576C3E57694035041
:101726000280C6D15B0575E5741490009F93F80896
:10173600C3E57598500280AED15BD15B0574C3E5F5
:1017460074940A5002809C120EADB184C2AF75EF3C
:0317560012D15B52
:0319FD00020FFDD9
:101A00000E0615FFFFFFFF03040A0101015AA5019D
:101A1000FFFFFFFFFF03FFFFFF25D0FAFA04FF01DE
:091A2000007AFF0101000300FF40
:101A400023585031384123202020202020202020DE
:101A500023424C48454C4923463333302320202031
:101A60002020202020202020202020202020202076
:101C0000C2AFC2D353D9BF7581C043B20343FF8073
:101C1000752438752503B1C975EF0275E24043F1AB
:101C20008053A47F75D4FFD2877DFA780379E67C50
:101C300010752200752300901DD67B0675249875BB
:101C400025013087028142208708D8FBD9F9DCF7CB
:101C500081B4308708D8FBD9F9DCF781B4B189E4C5
:101C600093A3C39A6004DDC381B4DBDBB17B600264
:101C7000812B7B08E493FAA3B15CDBF87A30B15C8A
:101C8000752200752300B17BEAFCEBFDC3ED94FEE9
:101C9000400EB17B8A278B28ED30E0048A828B834B
:101CA000B17B7AC270D8C3ED94FE601350CEBD00F4
:101CB00025EC60097520007521FF0200008100A855
:101CC00027A9280809D804D90281D3B17FEA89AAB3
:101CD000F281C50D81A0C3ED94035049EDA2E092BD
:101CE000007AC5C3E5829400E583941C50902000DF
:101CF00010438F02438F0175B7A575B7F1F030001F
:101D00001FA827A9280809438F01538FFDD804D99C
:101D100002A12089AAE275B7A575B7F1F0A3A10DBC
:101D2000538FFC817C7AC1BD030CE493A3FAB140CC
:101D3000DCF8B138817C817EAA22AB23B15CEBFA5E
:101D4000EA6222752608C3E52313F523E52213F57D
:101D50002250066323A0632201D526EAB1C9B1C986
:101D600075260AEAF4200102D287300102C287B147
:101D7000C9C3134002C201D526EB22B17FEAFB2082
:101D80008702A17F308702A184752608AE24AF2583
:101D9000C3EF13FFEE13FEB1CDB1C9C3EA13308711
:101DA000024480FA30E703632201C3E52313F523DD
:101DB000E52213F52250066323A0632201D526D91C
:101DC000E52265236523F52222AE24AF250E0FDE22
:101DD000FEDFFCD20122424C48656C693437316326
:041DE000F3300601D5
:00000001FF
